:020000040000FA
:06000000AEEF03F0120058
:0600080004EF04F01200F9
:060018000CEF04F01200E1
:02002A000000D4
:04002C000001746BF0
:100030001E0E716E0401400E096F200E0A6F040E31
:100040000B6F880E086F0401200E0E6F040E0F6FE9
:10005000400E0C6F1200550EA76EAA0EA76EA68258
:1000600012000401226B010E236F12000001726B5B
:10007000FDD80AE208D90800F5CF73F00001EFD8E7
:1000800073C0EFFF722BF4D7F86A1200F00E040170
:100090002217840EA66E0001726BE8D80AE2EBD834
:1000A0000F0E000172150F0801E1D5DF0001722B60
:1000B000F4D71200940EA66E0001726BD7D811E22D
:1000C0007251006E016A060ED89000360136E804BF
:1000D000FBE1026A01BE0268B3D8BDDF0001722BEA
:1000E000EDD7F86A1200A66A0001726BBFD80BE266
:1000F0000401225100017225A96EA680B0D8A8CFB4
:10010000EFFF722BF3D712000001726BAFD810E231
:100110000401225100017225A96EA1D8EF50A86EEA
:10012000040EA66E98DFA6B2FED70001722BEED7A2
:100130001200C40EA66E0001726B98D805E29BD81F
:100140008ADF0001722BF9D7F86A1200060E00014F
:10015000775D03E36D50020B01E071D0000174057F
:1001600011E104010CBF0DD00401400E096F400ED7
:10017000040108170401087D880E0401081300011A
:10018000746B5DD0040108BF5AD00001726B04018A
:100190002051FF0A34E0F80A2DE0020A26E0010AA5
:1001A0001FE0070A18E0010A11E0030A0AE0070A43
:1001B00008E0060A01E032D054DF0001040E726F3D
:1001C0002ED054DF050E0001722729D05FDF000119
:1001D000010E726F24D06EDF0001010E726F1FD00E
:1001E00082DF050E000172271AD08EDF0001010E9A
:1001F000726F15D09EDF0001010E726F10D06D96E8
:100200000001756B766B00017507000E765B0001CF
:100210007551761101E0F7D7FF0001D000D0000141
:10022000010E746F000172510AE072C00DF4400EAD
:1002300004010C1704010C7D880E04010C1312003C
:10024000040122510024F36E23510120F46E245145
:100250000220F86EF4CFF7FFF3CFF6FF12007251D1
:10026000EA6A250FE96E040EEA2212000401215108
:100270000001725D1200F3DFEFCF03F004D803C07A
:10028000F5FF0C00120072C000F0016A026A20EF54
:0202900001F07B
:0E0292006C5002E0000E01D0010E00090BE0DE
:1002A000040100513C0BE842E8420D0802E164EF12
:1002B00001F06EEF01F06C5002E0000E01D0010E73
:1002C000040901E01AD81200D5D800016A6B6B6BE3
:1002D000706B716B45EC02F084D8D2D0020E000135
:1002E0006A5D09E15CD8040100BD02D0C80E01D0EE
:1002F000880E006F12002AEF02F0040E0001775DF5
:1003000009E112C46EFF6E50000802E2050E01D032
:10031000030E776F00016A0509E10AD8040104BDE4
:1003200002D0C80E01D0880E046F12002AEF02F02E
:10033000A1D80001080E705D000E715903E270C073
:10034000DFFF02D0080EDF6EDFCF05F4DF50016A59
:10035000E850705F0150715B180E6E6F040E6F6F86
:10036000DF501CE0000178A307D06CC0F6FF6DC021
:10037000F7FF0800F55005D06CC0E9FF6DC0EAFF3B
:10038000EF506EC0E9FF6FC0EAFFEF6E00016C2B0B
:10039000000E6D236E2B6F23DF06E2D771D06AD873
:1003A00001C4DFFFDF5000017025706F000E712166
:1003B000716F180E6C6F040E6D6FDF5011E06CC022
:1003C000E9FF6DC0EAFFEF506EC0E9FF6FC0EAFFC2
:1003D000EF6E6E2B000E6F236C2B6D23DF06EDD7B7
:1003E0004FD000016B5105E13DD8840E006F040130
:1003F0001DD0040110AF1CD0000170510401165D26
:10040000000171510401175904E216C470F017C4B9
:1004100071F08EDF0001010E6A6F24D8800E006F2C
:100420000401180E066F040E076FC80E046F10D07B
:100430000001020E6A6F0401056BC80E046F04010F
:10044000080E016F180E026F040E036FC80E006FC6
:100450006D98120000016A6B05D8880E006F0401C8
:10046000046B12000401080E016F100E026F040EDF
:10047000036F1200D9CFE6FFE1CFD9FFE652120099
:0A048000E552E552E7CFD9FF120064
:06048A0004011051600B9B
:10049000E842E842E842E842E842000901E012008E
:1004A0001151080A39E0010A35E00F0A0AE0030A8F
:1004B00001E012000001010E6B6F0001040E776F66
:1004C00012000001010E6B6F0401130507E100012A
:1004D000060E6C6F070E6D6F120E13D0020E135DB9
:1004E00007E10001180E6C6F070E6D6F200E09D02A
:1004F000030E135D0AE10001380E6C6F070E6D6F7D
:10050000040E0001706F716B02D000016B6B000173
:10051000788312009AEF02F00001010E6B6F000168
:10052000790E6C6F000E6D6F000178930001010E63
:10053000706F12000001010E6B6F12C479F004019C
:10054000125104E10001050E776F12000001060E42
:06055000776F16EF00F0CA
:0A055600080E6D6E6DBAFED7686ADC
:10056000110E696E0001020E776F12006850040BC5
:1005700006E06950040B03E06D926994689468503A
:10058000010B04E06950010B01E027D86850100B03
:1005900009E06950100B06E0698468986D82A08AB2
:1005A0000300A19A6850200B09E06950200B06E077
:1005B00070A003D02AEC02F07090689A030E00013C
:1005C000775D01E209D06850080B06E06950080B1E
:1005D00003E049EC01F068961200686A7B0E696ED0
:1005E0006E6A160E706E68A602D06896FCD76D987B
:1005F0002AEC02F00001796B0001030E776F120004
:100600002A0EF66E000EF76E000EF86E000109005D
:10061000F550656F0900F550666F03E1656701D01D
:100620003DD00900F550606F0900F550616F090079
:10063000F550626F09000900F550E96E0900F550A8
:10064000EA6E090009000900F550636F0900F550D2
:10065000646F09000900F6CF67F0F7CF68F0F8CFB4
:1006600069F060C0F6FF61C0F7FF62C0F8FF0001EB
:10067000635302E1645307E00900F550EE6E63072F
:10068000F8E26407F9D767C0F6FF68C0F7FF69C0F2
:0E069000F8FF00016507000E665BBFD7120081
:02069E00926860
:1006A0009368FC0E946E806A040E816E826AD56A2D
:1006B000CD6ACA6AB16A070EB46EBD6ABA6AF16AD7
:1006C00082B402D000EF04F0140E6F6EABEC02F0B7
:1006D00082808282829000017B6BB6EC02F0A6ECF5
:1006E00000F000017B510001775D0BE0060E000178
:1006F0007B5D07E077C07BF0060E0001775D01E1CE
:060700008292EBD712000B
:0A0706001201000200000008D804F0
:100710000B00000000000001090220000101008020
:100720003209040000020000000007050102400039
:0C073000000705810240000004030904DA
:04073C00000EF36E4A
:1007400000EE00F0080E01D81200EA6002D0EE6A56
:0C075000FCD7F350E9601200EE6AFCD701
:04075C0013EE00F0A8
:1007600023EE00F0F86A059C00EC03F0BCEC03F00B
:080770004FEC03F0FBD712006F
:0207780012006D
:020000040030CA
:0100000024DB
:010001000EF0
:0100020038C5
:0100030018E4
:01000500807A
:010006008079
:010009008076
:01000B00A054
:00000001FF
